:020000040800F2
:10000000C806002091010008010D0008F90C000845
:10001000FD0C000841080008E3190008000000007A
:10002000000000000000000000000000491100086E
:10003000650A000800000000B90D00080912000858
:10004000AB010008AB010008AB010008AB010008E0
:10005000AB010008AB010008670A0008AB0100080B
:10006000AB010008AB010008AB010008AB010008C0
:10007000AB010008AB010008AB010008AB010008B0
:10008000AB010008AB010008AB010008AB010008A0
:10009000AB010008AB010008AB010008AB01000890
:1000A000AB010008AB010008AB010008AB01000880
:1000B000AB010008AB0100088D120008AB0100087D
:1000C000AB010008AB010008AB010008AB01000860
:1000D000AB010008B9170008AB010008AB0100082C
:1000E000AB010008AB010008AB01000800F002F80A
:1000F00000F03EF80AA090E8000C82448344AAF184
:100100000107DA4501D100F033F8AFF2090EBAE881
:100110000F0013F0010F18BFFB1A43F0010318473B
:100120006C2300008C230000103A24BF78C878C1EB
:10013000FAD8520724BF30C830C144BF04680C60ED
:10014000704700000023002400250026103A28BF35
:1001500078C1FBD8520728BF30C148BF0B60704739
:100160001FB59DE8030000F001F91FBD10B510BDDB
:1001700000F068F91146FFF7F3FF02F093F800F082
:10018000A7F903B4FFF7F2FF03BC02F083F8000005
:100190000948804709480047FEE7FEE7FEE7FEE71B
:1001A000FEE7FEE7FEE7FEE7FEE7FEE70448054957
:1001B000054A064B7047000029120008ED000008B0
:1001C000C8000020C8060020C8020020C802002085
:1001D000704700000EB5054614460E4612A000F00A
:1001E0009BF8284600F098F815A000F095F83046E6
:1001F00000F092F814A000F08FF800218DF80B1099
:100200000A210DF10A008DF80A1007E0224694FB3E
:10021000F1F401FB1422303200F8012D002CF5DC42
:1002200000F07AF800F070F82A2A2A2061737365CA
:100230007274696F6E206661696C65643A200000B3
:100240002C2066696C6520002C206C696E6520008E
:1002500010B5203AC0F00B80B1E81850203AA0E861
:100260001850B1E81850A0E81850BFF4F5AF5FEA95
:10027000027C24BFB1E81850A0E8185044BF18C948
:1002800018C0BDE810405FEA827C24BF51F8043BEF
:1002900040F8043B08BF7047D20728BF31F8023B43
:1002A00048BF11F8012B28BF20F8023B48BF00F8D7
:1002B000012B704770477047704770B50446051FA3
:1002C00000F034F80068002C14BF446870BD002CA6
:1002D00018BFAC423CBF20466468F8D301680A18D6
:1002E000AA4218BF456003D12A680546114401603F
:1002F00028684119A1421CBF6C6070BD61686960CB
:1003000021680844286070BD002000F08DF8FFF7D8
:100310002DFF012001F0BEFF10B5044602E0641C71
:1003200001F0BAFF20780028F9D110BD00487047CD
:100330006C0000200048704798000020704770470C
:100340007047704738B504460A4600206946AFF347
:100350000080002808BF38BD02460099204600F002
:100360009DF8012038BD012000F0D6B8F8B5AFF3F4
:100370000080054600200C46102000BF0646A81944
:10038000A0420DD9324669460020AFF30080070035
:1003900008BF00F0C1F80098A04218BF0546C41974
:1003A000FFF7C4FF05600746F01D20F0070046195F
:1003B000284600F06CF8B44208BFF8BDA21B3146D5
:1003C0003868BDE8F84000F069B870B50646FFF738
:1003D000ADFF056806F10B0020F00704B4429CBF96
:1003E000002070BD2B466A68BAB11068A04210D3D5
:1003F00004F1080188423CBF5068586007D3516837
:10040000101941601168091B016058601460101DCB
:1004100070BD13465268002AE7D121462846FFF7EF
:1004200091FF0028DED170BD10B500F05DF8BDE889
:10043000104000F053B800F076B800000048704754
:10044000640000207546FFF7F9FFAE4605006946D7
:10045000534620F00700854618B020B5FFF7A6FEEA
:10046000BDE820404FF000064FF000074FF00008B5
:100470004FF0000B21F00701AC46ACE8C009ACE836
:10048000C009ACE8C009ACE8C0098D46704700213E
:100490000160C0E9011070471020704703464068B2
:1004A0008C46002818BF88423CBF03464068F8D3FA
:1004B00018681844884207D00CF1030020F00700A8
:1004C000001D411A521A0146081D0A60FFF7F5BEC9
:1004D0000446AFF300802046FFF753FE002801D00A
:1004E00001F0D8BE7047000010B5002102A000F056
:1004F00027F8012010BD0000534947414252543AA9
:100500002041626E6F726D616C207465726D696EF0
:100510006174696F6E00000010B500F02BF8BDE843
:100520001040FFF7DBBF10B500F04FF8016919B1BB
:1005300000220261884701E080688047FFF7E4FEFF
:1005400070B505460C460A2000E06D1C01F0A4FEC3
:1005500035B128780028F8D102E0641C01F09CFE37
:1005600014B120780028F8D1BDE870400A2001F0CD
:1005700093BE000010B5012805D0002103A0FFF7AD
:10058000DFFF012010BD09A1F8E7000053494752E1
:10059000544D454D3A204F7574206F662068656153
:1005A00070206D656D6F7279000000003A2048651B
:1005B0006170206D656D6F727920636F72727570F6
:1005C0007465640010B5FFF79FFE70B500F022F867
:1005D00004680546A4B92020FFF7F7FE040011D0F7
:1005E000094900202C60C4E900010849A16020737A
:1005F000206160610649A06109B100F00FF8E06177
:10060000204670BDFFF780FE00000000C505000811
:100610000000000000487047A000002010B58820AE
:10062000FFF7D3FE002801D00021017010BD802902
:1006300002D808B1017809B100207047012100F803
:10064000081B704718B100F10802914201D0002048
:10065000704700210170704721B1826842F00102A9
:10066000826003E0826822F001028260704700002D
:1006700010B504461248844208D10121401500F00B
:10068000E9FB0021601500F0E5FB17E00D4884420E
:1006900008D10121001500F0DDFB0021201500F03C
:1006A000D9FB0BE00848844208D10121C80300F0BF
:1006B000D1FB00214FF4004000F0CCFB10BD000046
:1006C0000024014000280140003C014021B1826823
:1006D00042F48012826003E0826822F48012826019
:1006E0007047014600208A6812F0040F01D00120F3
:1006F00000E0002070470146C86C80B27047024697
:10070000002013680B4201D0012000E00020704758
:10071000014600208A6812F0080F01D0012000E095
:100720000020704730B502460020002350680F4C6F
:100730002040D1E9004544EA0524204350609068F8
:100740000B4C2040D1E903542C438D6844EA450406
:1007500020439060D06A20F470000C7D641EE4B2E7
:10076000234340EA0350D06230BD0000FFFEF0FF9B
:10077000FDF7F1FFF0B504460D4600200021092DDC
:1007800011DDE068A5F10A0606EB4607072606FA22
:1007900007F18843A5F10A0606EB460603FA06F1BF
:1007A0000843E0600CE0206905EB4507072606FAE0
:1007B00007F1884305EB450603FA06F1084320617B
:1007C000072A0FDA606B561E06EB86071F2606FA0D
:1007D00007F18843561E06EB860605FA06F1084324
:1007E000606322E00D2A0FDA206BD61F06EB860726
:1007F0001F2606FA07F18843D61F06EB860605FA80
:1008000006F10843206310E0E06AA2F10D0606EB52
:1008100086071F2606FA07F18843A2F10D0606EBAC
:10082000860605FA06F10843E062F0BD816841F0F2
:10083000080181607047816841F004018160704760
:1008400000BFFEE739B1084A1268012383401A430A
:10085000054B1A6006E0044A1268012383409A435C
:10086000014B1A60704700000074004010B5012170
:10087000480700F0CFFA00214FF0005000F0CAFA0C
:1008800010BD000030B5002200230A4C226840F65B
:10089000FE748440A243D1E900452C438D682C436B
:1008A000CD6844EA050303FA00F42243014C2260B8
:1008B00030BD00000074004008B500220092054AD7
:1008C000009200F10802009B1A440092009A116005
:1008D00008BD00000074004008B500220092054ADF
:1008E000009200F11402009B1A440092009A1160D9
:1008F00008BD00000074004029B1064A5268024356
:10090000044B5A6004E0034A52688243014B5A6028
:1009100070470000002004E0016821F0010101603F
:100920000021016041608160C1604C49884208D16A
:100930004A490839496841F00F01484A083A51606C
:100940008AE046491431884208D144490839496847
:1009500041F0F001414A083A51607DE03F492831B9
:10096000884208D13D490839496841F470613B4AE1
:10097000083A516070E039493C31884208D1374922
:100980000839496841F47041344A083A516063E0DB
:1009900032495031884208D130490839496841F418
:1009A00070212E4A083A516056E02C496431884241
:1009B00008D12A490839496841F47001274A083AA0
:1009C000516049E025497831884208D123490839E6
:1009D000496841F07061214A083A51603CE0204981
:1009E000884206D1011F096841F00F01021F116002
:1009F00032E01B491431884208D11949091F09689E
:100A000041F0F001164A121F116025E01449283107
:100A1000884208D11249091F096841F47061104ADF
:100A2000121F116018E00E493C31884208D10C4970
:100A3000091F096841F47041094A121F11600BE057
:100A400007495031884207D10549091F096841F417
:100A50007021034A121F1160704700000800024015
:100A600008040240704710B501F0A4F8012000F01E
:100A700001F810BD014908607047000014040140EE
:100A800000212349C268002A3AD00A461268036846
:100A90009A430B461A600A1D126803689A430B1D9D
:100AA0001A60426811440A6803681A430A60184AC7
:100AB0000832126803689A43154B08331A601A1DEE
:100AC000126803689A43124B0C331A608268102A2A
:100AD0000ED11A1F126803681A430D4B08331A60AF
:100AE0001A1D126803681A43094B0C331A600DE093
:100AF0000749826811440A6803681A430A6005E0DE
:100B0000426811440A6803689A430A60704700000B
:100B10000004014030B500228B071C0F0F2303FA9D
:100B200004F20B4B8C1053F824309343084C8D1077
:100B300044F8253023468C1053F824308C07240FBA
:100B400000FA04F42343024C8D1044F8253030BDE4
:100B5000080001402DE9F041024600250026002052
:100B600000230024002791F808C00CF00F0591F82D
:100B700008C01CF0100F03D0D1F804C04CEA0505E2
:100B800091F800C0BCF1000F31D0146800202BE0B8
:100B90004FF0010C0CFA00F3B1F800C00CEA0306A8
:100BA0009E4220D183004FF00F0C0CFA03F7BC4398
:100BB00005FA03FC4CEA0404D1F808C0BCF1280F84
:100BC00006D14FF0010C0CFA00FCC2F814C00AE088
:100BD000D1F808C0BCF1480F05D14FF0010C0CFA58
:100BE00000FCC2F810C0401C0828D1D31460B1F832
:100BF00000C0BCF1FF0F34DD546800202EE000F18E
:100C0000080C4FF0010808FA0CF3B1F800C00CEA28
:100C100003069E4221D183004FF00F0C0CFA03F71C
:100C2000BC4305FA03FC4CEA0404D1F808C0BCF14B
:100C3000280F05D100F1080C08FA0CF8C2F814804E
:100C4000D1F808C0BCF1480F07D100F1080C4FF0F3
:100C5000010808FA0CF8C2F81080401C0828CED30E
:100C60005460BDE8F0810000F0B50A46002300247E
:100C70000021002500F00046B6F1004F02D11D4EC4
:100C8000F16901E01B4E7168C0F3034583B200F4C3
:100C90004016B6F5401F08D121F07061154E7668F8
:100CA00026F07066134F7E6012E000F48016B6F5F1
:100CB000801F06D1032606FA05F4A14341F07061B6
:100CC00006E0460D360103FA06F6B14341F07061C5
:100CD00022B1460D360103FA06F6314300F0004614
:100CE000B6F1004F02D1034EF16101E0014E716097
:100CF000F0BD00000000014000BFFEE700BFFEE7BE
:100D000000BFFEE770B5002100230F2244680CB33A
:100D1000164C246804F4E064C4F5E064210AC1F1CF
:100D20000403CA40447804FA03F184781440214350
:100D300009010F4C0678A155047804F01F05012421
:100D4000AC4005786D114FF0E02606EB8505C5F83F
:100D5000004109E0047804F01F050124AC40054D72
:100D60000678761145F8264070BD00000CED00E0D5
:100D700000E400E080E100E010B5024600200C4BEA
:100D8000186820F00300104318600A4B1B6843F0FA
:100D90000403084C2360012901D130BF00E020BFCB
:100DA000044B1B6823F00403024C236010BD0000B9
:100DB0000070004010ED00E0704700000146002088
:100DC000034A506820F440400843506070470000D8
:100DD0000010024029B1064A52690243044B5A618D
:100DE00004E0034A52698243014B5A617047000094
:100DF0000010024029B1064AD2690243044BDA616D
:100E000004E0034AD2698243014BDA617047000073
:100E10000010024029B1064A12690243044B1A61CC
:100E200004E0034A12698243014B1A6170470000D3
:100E30000010024029B1064A92690243044B9A61AC
:100E400004E0034A92698243014B9A6170470000B3
:100E50000010024029B1064AD2680243044BDA600E
:100E600004E0034AD2688243014BDA607047000015
:100E70000010024070B5002100230024002200254C
:100E80002C4E766806F00C0121B1042905D0082902
:100E900021D105E0284E066020E0274E06601DE0C7
:100EA000244E766806F47013224E766806F4803479
:100EB000022606EB93431CB9204E5E43066009E010
:100EC0001C4EF66A06F00F06751C1B4EB6FBF5F6B7
:100ED0005E43066002E0184E066000BF00BF154E7C
:100EE000766806F0F0010909154E725C0668D64076
:100EF0004660104E766806F4E061090A104E725C96
:100F00004668D64086600B4E766806F46051C90A82
:100F10000B4E725C4668D640C660064E766806F494
:100F20004041890B074E725CC668B6FBF2F606615B
:100F300070BD00000010024000127A0000093D0060
:100F4000430000205300002010B50146002200237A
:100F500000204A11012A02D1094C236806E0022A26
:100F600002D1074C236A01E0054C636A01F01F02BD
:100F7000012494401C4201D0012000E0002010BD5B
:100F8000001002400248406800F00C00704700006A
:100F9000001002401149096821F480310F4A1160A4
:100FA0001146096821F480211160B0F5803F03D01B
:100FB000B0F5802F0ED106E00849096841F4803170
:100FC000064A116007E00549096841F4A021034A77
:100FD000116000E000BF00BF704700000010024039
:100FE00001490866704700000000424201460020A7
:100FF000034A506820F00300084350607047000027
:101000000010024038B5002000900024002500BFE9
:101010003120FFF799FF05460098401C009000988A
:10102000B0F5A06F01D0002DF2D03120FFF78CFF7A
:1010300008B1012400E00024204638BD3EB5044636
:101040000A4951F824000121FFF7F4FE084830F85E
:101050001400ADF800001020029003200190054913
:1010600051F824006946FFF775FD3EBD18240008BD
:101070001424000800000020034931F81010034A2E
:1010800052F820205161704714240008000000200D
:10109000034931F81010034A52F8202011617047BB
:1010A000142400080000002030B589B004460D4625
:1010B0001E4951F8241041F001000121FFF7BAFE4A
:1010C000042008901A4830F81400ADF818001949A7
:1010D00051F8240006A9FFF73DFD012D23D1164A42
:1010E00012F81410154A12F81400FFF713FD1448F3
:1010F00030F8140002900020039008200490012092
:10110000059002A8FFF7BCFC0E4810F814008DF8FB
:1011100000000F208DF801008DF8020001200190E1
:101120006846FFF7EFFD09B030BD00002824000835
:10113000242400080800002020240008222400089D
:101140002C2400082E240008704710B500F002F887
:1011500010BD00000CB500200190009029480068E7
:1011600040F480302749086000BF2648006800F43A
:10117000003000900198401C0190009818B9019827
:10118000B0F5A06FF1D11F48006810F4003F02D005
:101190000120009001E0002000900098012830D14B
:1011A0001848406817494860084640684860084643
:1011B000406848600846406820F47C104860084653
:1011C000406840F4981048600846006840F080701D
:1011D000086000BF0B48006810F0007FFAD0094893
:1011E000406820F00300074948600846406840F026
:1011F0000200486000BF0348406800F00C00082867
:10120000F9D10CBD0010024010B506480078012845
:1012100003D10020FFF73CFF02E00020FFF72CFF86
:1012200010BD00004200002010B51448006840F0D6
:1012300001001249086008464068114908400F49FA
:101240004860084600680F4908400C490860084695
:10125000006820F4802008600846406820F4FE0002
:1012600048604FF41F0088600020C862FFF76DFFE0
:101270004FF000600449086010BD000000100240FB
:101280000000FFF8FFFFF6FE08ED00E010B50221B8
:10129000074800F02DF948B10221054800F016F882
:1012A00000F0A6FD0021024800F013F810BD000078
:1012B0000008004021B1028842F08002028004E070
:1012C00002884FF67F731A4002807047CA43028239
:1012D000704721B1028842F00102028004E00288D6
:1012E0004FF6FE731A400280704731B1B0F84420C7
:1012F00042F40042A0F8442005E0B0F84420C2F3D4
:101300000E02A0F84420704710B504466848844295
:1013100008D10121C014FFF79DFD0021E014FFF763
:1013200099FDC4E0B4F1804F08D101210846FFF7D0
:1013300071FD00210120FFF76DFDB8E05D4884429A
:1013400008D101210220FFF765FD00210220FFF7EF
:1013500061FDACE05848844208D101210420FFF728
:1013600059FD00210420FFF755FDA0E053488442B9
:1013700008D101210820FFF74DFD00210820FFF7CB
:1013800049FD94E04E48844208D101211020FFF726
:1013900041FD00211020FFF73DFD88E049488442CF
:1013A00008D101212020FFF735FD00212020FFF783
:1013B00031FD7CE04448844208D101214014FFF70C
:1013C00049FD00216014FFF745FD70E03F4884426D
:1013D00009D10121C804FFF73DFD00214FF4002091
:1013E000FFF738FD63E03A48844209D1012108053E
:1013F000FFF730FD00214FF48010FFF72BFD56E082
:101400003448844209D101214805FFF723FD00211A
:101410004FF40010FFF71EFD49E02F48844208D129
:1014200001214020FFF7F6FC00214020FFF7F2FCED
:101430003DE02A48844208D101218020FFF7EAFCE0
:1014400000218020FFF7E6FC31E02548844208D1E6
:1014500001218015FFF7DEFC0021A015FFF7DAFC63
:1014600025E02048844209D101210804FFF7F2FC5D
:1014700000214FF48030FFF7EDFC18E01A48844259
:1014800009D101214804FFF7E5FC00214FF40030A9
:10149000FFF7E0FC0BE01548844208D101218804E5
:1014A000FFF7D8FC00214FF48020FFF7D3FC10BDDC
:1014B000002C01400004004000080040000C0040E7
:1014C000001000400014004000340140004C014076
:1014D000005001400054014000180040001C004032
:1014E000002000400040014000440140004801400D
:1014F00030B50246002000230024158A05EA0103C6
:10150000958905EA010413B10CB1012000E0002027
:1015100030BD1AB183890B43838102E083898B43F9
:101520008381704770B5002400220023058C4FF69C
:10153000FE7635400584028C8388048B4FF68F75C8
:101540002C40B51E2C400D882C43751E2A400D8959
:101550002A434D882A43144DA8420BD0134DA8426C
:1015600008D0134DA84205D0124DA84202D0124D0A
:10157000A84213D14FF6F7752A404D892A434FF6FA
:10158000FB752A408D882A434FF6FF652B404FF6A6
:10159000FF552B408D892B43CD892B4383800483BA
:1015A000CD888586028470BD002C01400034014046
:1015B00000400140004401400048014070B5002453
:1015C00000220023058C4FF6EF7635400584028C0F
:1015D0008388048B48F6FF752C404FF6FF452C405E
:1015E0000D884FF6FF7606EA05252C434FF6DF758A
:1015F0002A400D8906EA05152A434D8806EA051595
:101600002A43154DA84202D0144DA8421DD14FF6D1
:101610007F752A404D894FF6FF7606EA05152A4365
:101620004FF6BF752A408D8806EA05152A434FF606
:10163000FF352B404FF2FF752B408D8906EA85055B
:101640002B43CD8906EA85052B4383800483CD880F
:101650000587028470BD0000002C01400034014069
:1016600070B5002200230024058C4EF6FF7635402D
:101670000584038C8488828B48F6FF752A404FF6D8
:10168000FF452A400D884FF6FF7606EA05252A43D6
:101690004DF6FF752B400D8906EA05352B434D8825
:1016A00006EA05352B430B4DA84202D00A4DA8424D
:1016B00008D14BF6FF752C408D894FF6FF7606EA70
:1016C00085152C4384808283CD88A0F84050038404
:1016D00070BD0000002C0140003401400A4600218A
:1016E000818B4FF2FF7319404FF6FF7303EA022319
:1016F00019438183704781857047A0F84010704777
:10170000002202881D4B98420ED01D4B98420BD0F0
:10171000B0F1804F08D01B4B984205D01A4B98422D
:1017200002D01A4B984204D14FF68F731A404B885F
:101730001A43174B984207D0164B984204D04FF6E5
:10174000FF431A40CB881A4302808B8883850B881D
:1017500003850A4B98420BD0094B984208D00E4B98
:10176000984205D00D4B984202D00D4B984201D1C2
:101770000B7A03860123838270470000002C01400E
:10178000003401400004004000080040000C00400C
:10179000001000400014004000400140004401409F
:1017A000004801404FF6FF71818000210180C18017
:1017B000418001727047000010B51148008810F098
:1017C000200F1BD00E48008820F020000C49088014
:1017D000091D0988CAB20B490868411C094B1960E8
:1017E00009490A54712A09D100201946086032219A
:1017F000034800F0E7F801200449087010BD00001C
:101800000038014010000020580000200C0000208B
:1018100010B502460020108A4FF2FF0318400B88D3
:101820004C8823438C882343CC882343184310825D
:1018300010BD0021018041808180C180704721B1AD
:10184000828942F40052828104E082894DF6FF735E
:101850001A40828170471AB1838A0B43838202E067
:10186000838A8B438382704702460020B1F5007F54
:1018700000D100BF13880B4201D0012000E00020FE
:101880007047F0B503460024002600250020A1F58E
:1018900010676A3F00D100BF1846C1F3421401F03F
:1018A0001F06012707FA06F5012C01D10C3004E0D0
:1018B000022C01D1103000E014301AB107682F4318
:1018C000076002E00768AF430760F0BD2DE9F0470D
:1018D00086B005460E460024A24600BFA14600275A
:1018E000B08900B100BF2F462C8A4CF6FF7004402F
:1018F000F08804432C82AC894EF6F3100440B08883
:1019000031890843718908430443AC81AC8A4FF69E
:10191000FF400440B0890443AC8201A8FFF7AAFA53
:101920001F48874202D1DDF810A001E0DDF80CA0CD
:10193000A88910F4004F08D00AEBCA0000EB0A1087
:1019400031684900B0FBF1F807E00AEBCA0000EB90
:101950000A1031688900B0FBF1F86420B8FBF0F0A0
:1019600004012009642101FB1089A88910F4004FAB
:1019700008D0322000EBC900B0FBF1F000F0070006
:10198000044308E0322000EB09106421B0FBF1F0C1
:1019900000F00F0004432C8106B0BDE8F087000082
:1019A00000380140C1F30802828070474FF416519D
:1019B000016000218180C18001810C2141810021D1
:1019C0008181704730B505460C46E1B22846FFF7E5
:1019D000E9FF00BF80212846FFF746FF0028F9D025
:1019E00030BD00BFFEE700002DE9F35F044600BFF5
:1019F000A0888246002704F11000019900F070FCD5
:101A0000002522E02E46A088B04200D904E07E22C4
:101A100013A11BA0FEF7DEFB206830F916008346F9
:101A200000BFA269911EA161B2F900002269A169FB
:101A3000914205D2A28A216901EB4201891EA1616E
:101A400000BF81460BFB09776D1C5545DAD300BFFB
:101A50000F2047FA00F00FFA80F84046BDE8FC9FDF
:101A60002E2E5C2E2E5C2E2E5C6F7064726163686D
:101A700074315C6473626B6C617373656E2E6800A5
:101A8000696E646578203C2061616E74616C000051
:101A90002DE9F04704460E46174625461FFA86F8FC
:101AA000B946C5F80090A5F804800020A871286800
:101AB000A8602868E860B8F1000F00D004E0332285
:101AC00007A10FA0FEF786FB00BF2C46B1B204F1C0
:101AD000100000F03BFCA0F110042046BDE8F087A8
:101AE0002E2E5C2E2E5C2E2E5C6F706472616368ED
:101AF00074315C6473626B6C617373656E2E680025
:101B00006120213D2030000004460321204600F0E2
:101B1000C3F8012104F5847000F03CFA00BF04F51D
:101B2000847000F06FFB05B2294604F58A70FFF758
:101B30005BFF00F5006086B2314604F5827000F06C
:101B400071FBECE770B504460121204600F05CF91A
:101B500004460A4820600A4A1F2104F58A70FFF7EC
:101B600097FFA0F58A7442F210756426642104F58B
:101B7000847000F08BF9204670BD000074240008CA
:101B8000D423000870B50446094804F58A7520601E
:101B900004F5927000F014FCA0F11005284600F046
:101BA0000FFCA0F58A74204600BF044670BD0000FB
:101BB000742400080120014908707047400000208B
:101BC00070B504460D46204600F018F92946204617
:101BD00000F001F870BD70B505460C46012C07D128
:101BE00002210120FFF7C8F8284600F0E1F802E0E2
:101BF00000BF00BF30BF70BD10B58AB004460121E0
:101C00000220FFF7F7F84FF40070ADF8000018203D
:101C100002900220019069461C48FEF79BFF0121BB
:101C20001B48FFF721F81B48FFF76EFB42F6E06008
:101C3000ADF820004FF47A70ADF81C000020ADF82C
:101C40002200ADF81E0007A91248FFF759FD6020D9
:101C5000ADF80C000120ADF80E0041F27070ADF847
:101C600012000020ADF8140003A90A48FFF7F8FCA1
:101C700008210848FFF732FD01210648FFF71AFB4B
:101C800001210448FFF725FB0AB010BD00100140F8
:101C9000000C1A000004004070B506460C46052CE6
:101CA00000DA05E04FF49B720DA118A0FEF792FA3E
:101CB00024B900211C48FFF70CFB10E01B4830F84A
:101CC000145001211848FFF704FB6804010C164862
:101CD000FFF711FD29461448FFF70FFD00BF70BD47
:101CE0002E2E5C2E2E5C53544D3332564C44697369
:101CF000636F766572795C73746D3332436F6E74A3
:101D0000726F6C6C65722E63707000007374616E1C
:101D1000643C4B6E69707065724C45445F4C616108
:101D20007473746500000000000400406024000823
:101D300010B58AB0044601210420FFF75BF81B4868
:101D4000FFF7E2FA4FF6FF70ADF8200042F6E060D0
:101D5000ADF81C000020ADF82200ADF81E0007A968
:101D60001248FFF7CDFC1020ADF80C000120ADF8B3
:101D70000E000020ADF8140003A90C48FFF7D2FBB9
:101D80001E208DF8040000208DF8060004208DF838
:101D900005000120029001A8FEF7B4FF01220221F4
:101DA0000248FFF7B6FB0AB010BD00000008004073
:101DB00010B504464FF48030FFF7ECF8FFF722F936
:101DC000C4F81001D4F8100101280FD1FFF708F969
:101DD00000BF3920FFF7B8F80028FAD00220FFF73B
:101DE00005F900BFFFF7CEF80828FBD110BD0000B1
:101DF0000120014908707047410000200021014A7C
:101E0000117070474000002070B504460D461E4812
:101E100020602146201D00F087F9041F002229467A
:101E200004F5827000F03EF9A0F58274052229467F
:101E300004F5847000F0B8F8A0F5847472B6002040
:101E4000FFF7FCF80020FFF717F90120FFF7F6F87D
:101E50000120FFF711F901210020FFF725F90121E9
:101E60000846FEF749FD01210220FEF745FD01214C
:101E7000C802FEF741FD2046FFF75AFF2046FFF754
:101E8000BBFE62B6204670BD8424000830B587B022
:101E900004460D464FF6FF70854200D205E040F241
:101EA0009D1216A11FA0FEF795F9A58004A8FFF7C3
:101EB00079FCA088ADF814001820ADF810000020BF
:101EC000ADF81600ADF8120004A92068FFF718FC61
:101ED0006020ADF800000120ADF80200A088ADF848
:101EE00006000220ADF8080069462068FFF766FB8F
:101EF00001212068FFF7F9F907B030BD2E2E5C2EC6
:101F00002E5C53544D3332564C446973636F76657F
:101F100072795C73746D33325065726966732E63C7
:101F20007070000074733C363535333500000000A6
:101F300070B506460C464FF6FF70844200DA05E0A5
:101F40004FF4CA7206A110A0FEF744F94FF47A705C
:101F500004FB00F529463046FFF798FF70BD0000EE
:101F60002E2E5C2E2E5C53544D3332564C446973E6
:101F7000636F766572795C73746D33325065726924
:101F800066732E637070000074733C3635353335DC
:101F90000000000070B504460D462E46314620680C
:101FA000FFF797F970BD0000F0B589B005460C4603
:101FB00016464FF080402860AE8001214015FEF7A4
:101FC00039FF0020FEF7FAFE334A07CA06AB07C303
:101FD0000CB940200CE0012C01D1022008E0022CB9
:101FE00001D1042004E0042C01D1802000E0042071
:101FF000ADF8180006A92948FEF7ACFD0CB906207B
:102000000CE0012C01D1012008E0022C01D10220BA
:1020100004E0042C01D1072000E0022007462048FC
:10202000FEF726FB18221C490C316846FEF710F912
:1020300069461B48FEF776FB0723012239461848FC
:10204000FEF798FB01211648FEF740FB01210846E8
:10205000FEF7D0FEA9882846FFF76AFF0121104845
:10206000FEF7FAFA00212868FFF733F90C48FEF76B
:10207000DDFB00BF0A48FEF74BFB0028FAD10848F9
:10208000FEF7D9FB00BF0648FEF72BFB0028FAD16C
:10209000284609B0F0BD00003C24000800080140BB
:1020A0000024014070B588B005460C4616462C60E9
:1020B00001214807FEF79EFEFEF7D8FB124A07CA29
:1020C00005AB07C30CB9202000E01020ADF81400C8
:1020D00005A90E48FEF73EFD0020019002900390F6
:1020E00004900CB9102100E00021084601A9FEF778
:1020F000C9FB0CB9102100E0002108460121FEF7C0
:10210000A1FB284608B070BD30240008000801403B
:1021100070B504460D4621460248FFF753FC2046A1
:1021200070BD00000038014030B58BB004460D464C
:1021300004F1080060600020A4F8F800012084F891
:10214000FA00C4F8FC5001210846FEF743FE0121C5
:1021500044F20400FEF76EFE18200A904FF49050EF
:10216000ADF820000220099008A92348FEF7F2FCF0
:1021700048200A904FF44060ADF8200002200990FA
:1021800008A91D48FEF7E6FC02A8FFF752FB02A9CA
:102190001A48FFF73DFB04A8FFF708FC4FF4612045
:1021A00004904FF44070ADF81C0004A91348FFF7E9
:1021B0008DFB25208DF8000000208DF80200012005
:1021C0008DF8010001906846FEF79CFD012240F267
:1021D00025510A48FFF755FB012280210748FFF7E8
:1021E0003AFB0748FEF798FB01210448FFF727FB5D
:1021F00020460BB030BD000000080140003801400F
:102200004400024010B5044600BF02210448FEF716
:1022100076FA0028F9D00248FEF76DFA10BD0000EA
:102220000024014070B504460D46B5F5805F02DB21
:1022300040F6FF7000E028460646206820B9314687
:102240000020FEF749FB03E031460020FEF734FB97
:1022500070BD10B500F001F810BD10B5FEF72DF8F7
:1022600010BD10B500F002F810BD000010B504005C
:1022700007D1012405E0FEF75DF8006800B90448C5
:1022800080472046FEF7A1F80028F4D010BD0000DA
:102290003704000800BFFEE710B50446204600F0F2
:1022A00017F810BD00B5CDB06846FFF74BFC002114
:1022B0006846FFF7F1FC00216846FFF781FC68469D
:1022C000FFF722FC6846FFF75DFC00204DB000BD23
:1022D00010B50446E0B20021FFF71AFF10BD000060
:1022E00070B504460D46A079012800D104E05A22B9
:1022F00009A111A0FDF76EFFE068A060E168881CED
:10230000E0600D80A188206800EB4100E168884210
:1023100001D12068E06070BD2E2E5C2E2E5C2E2E2A
:102320005C6F70647261636874315C6473626B6C5F
:10233000617373656E2E680074727565203D3D2073
:1023400064796E416C6C6F63000000002DE9F04110
:1023500004460D466800FFF784FF2060A580012039
:10236000A0712068A0602068E06005B104E0202230
:1023700009A111A0FDF72EFFA688206800EB4600FA
:10238000871E00BF002027F80209701E0600F9D141
:102390002046BDE8F08100002E2E5C2E2E5C2E2EF5
:1023A0005C6F70647261636874315C6473626B6CDF
:1023B000617373656E2E68006120213D203000003E
:1023C00010B50446A079012802D12068FFF741FF2B
:1023D000204610BDBFFF3A00A300BEFF4CFED8FF51
:1023E0007103AB01CFFA7DFBE505180840FBDDF476
:1023F000D301550CD301DDF440FB1808E5057DFB46
:10240000CFFAAB017103D8FF4CFEBEFFA3003A0028
:10241000BFFF0000000200011000000010000000DB
:1024200000000000010000000400000001000600A0
:10243000000000000200000010000000000000008A
:102440000300000000000000000000000000000089
:102450000000000000000600000000000100000075
:102460000000E02E7017B80BE80300000000000029
:1024700000000000851B00080000000000000000B4
:10248000000000000000000000000000AC24000874
:102490000000002058000000280100080425000862
:1024A00058000020700600004401000800100140A0
:1024B0000010014000080140000000000000000082
:1024C000043801400000000010000000000000007F
:1024D000000000008000000000000000000000007C
:1024E00000000000002000000000000000000000CC
:1024F00000000001020304010203040607080902A8
:0425000004060800C5
:04000005080000ED02
:00000001FF
